:040000000200663262
:01000B0032C2
:0100130032BA
:01001B0032B2
:20002300322B2B2B2042617373706564616C2042502D312056312E32202F2041543839438C
:2000430032303531202843292053746566616E204861726173696D2030382F32303037201B
:200063002B2B2B758123C2D3C2D4758920758840758DFF75987C75A8007590FF75B0FF7519
:200083000C1E750800750900752000752100752200750B60C2B4E590D2B4540F4490F50AEF
:2000A3001200D812010312012E1201591201841201AF1201DA12020512023012025B12026A
:2000C300861202B11202DC12030712032412034112035C80CBC2B2E590D2B230E0102008C6
:2000E3000122C2082005FA750924120377222008F03004031203927508241203ABD208224E
:20010300C2B2E590D2B230E11020090122C2092005FA750925120377222009F03004031265
:2001230003927508251203ABD20922C2B2E590D2B230E210200A0122C20A2005FA7509265D
:2001430012037722200AF03004031203927508261203ABD20A22C2B2E590D2B230E31020E5
:200163000B0122C20B2005FA75092712037722200BF03004031203927508271203ABD20BD5
:2001830022C2B2E590D2B230E410200C0122C20C2005FA75092812037722200CF0300403C6
:2001A3001203927508281203ABD20C22C2B2E590D2B230E510200D0122C20D2005FA7509E2
:2001C3002912037722200DF03004031203927508291203ABD20D22C2B2E590D2B230E61050
:2001E300200E0122C20E2005FA75092A12037722200EF030040312039275082A1203ABD231
:200203000E22C2B2E590D2B230E710200F0122C20F2005FA75092B12037722200FF030042B
:200223000312039275082B1203ABD20F22C2B3E590D2B330E01020100122C2102005FA755E
:20024300092C120377222010F030040312039275082C1203ABD21022C2B3E590D2B330E1CD
:200263001020110122C2112005FA75092D120377222011F030040312039275082D1203AB63
:20028300D21122C2B3E590D2B330E21020120122C2122005FA75092E120377222012F030D1
:2002A300040312039275082E1203ABD21222C2B3E590D2B330E31020130122C2132005FA40
:2002C30075092F120377222013F030040312039275082F1203ABD21322C2B3E590D2B330AD
:2002E300E41020140122C2142005FA750930120377222014F030040312039275083012039B
:20030300ABD21422C2B4E590D2B420E60A30060122D206750B7F2220060122C206750B6063
:2003230022C2B4E590D2B420E70A30070122D207750B402220070122C207750B6022C2B476
:20034300E590D2B420E40830040122D204800620040122C2041203C422C2B4E590D2B42047
:20036300E50830050122D205800620050122C2051203C422850A993099FDC299850999302E
:2003830099FDC2997599003099FDC29971D922850A993099FDC2998508993099FDC29975C9
:2003A30099003099FDC29922850A993099FDC2998508993099FDC299850B993099FDC29984
:2003C300227424750923050912037704B431F775210075220022A90C09D901227AF8DAFEF2
:0603E3007AF8DAFE80F357
:0003E90113
